:100000001AC3000050C300004EC300004CC30000E0
:100010004AC3000048C3000046C3000044C30000B8
:1000200042C3000040C300000C949E2F0C94863005
:100030000C94532F38C3000036C3000034C30000B3
:1000400032C3000030C300002EC300002CC30000E8
:100050002AC300000C947A2F26C3000024C300009A
:1000600022C3000020C300001EC300001CC3000008
:100070001AC3000018C3000016C3000014C3000018
:1000800012C3000010C300000EC300000CC3000028
:100090000AC3000008C3000006C3000004C3000038
:1000A00002C3000000C30000FEC2000005010902F7
:1000B000A10185020901A1000509190129081500FE
:1000C0002501950875018102050109300931158165
:1000D000257F95027508810609381581257F9501D0
:1000E00075088106050C0A38021581257F95017572
:1000F000088106C0C005010980A101850319012AF4
:10010000B700150126B700950175108100C0050CD8
:100110000901A101850419012AA002150126A002E6
:10012000950175108100C005010906A1018506052C
:100130000719E029E71500250195087501810205D9
:1001400007190029EF1500250195F07501810205B9
:10015000081901290595057501910295017503910D
:1001600001C00660FF0961A1010962150026FF00B8
:100170009520750881020963150026FF00952075FA
:10018000089102C005010906A101050719E029E748
:1001900015002501950875018102950175088101F9
:1001A0000507190029FF150026FF0095067508812F
:1001B000000508190129051500250195057501910E
:1001C00002950175039101C00000000000000000CD
:1001D000000000000000000000000000000000001F
:1001E0000000000000000000000000007E0F00D4AE
:1001F000FFFFFFC7000000780000000000000000C3
:100200002A2B280000000000000000000000000071
:1002100000000029000000002C1E3420212224347C
:100220002627252E362D3738271E1F20212223244E
:1002300025263333362E37381F0405060708090AEA
:100240000B0C0D0E0F101112131415161718191A86
:100250001B1C1D2F3130232D350405060708090A04
:100260000B0C0D0E0F101112131415161718191A66
:100270001B1C1D2F3130354C09025B00030100A00F
:10028000FA09040000010301010009211101000124
:10029000224400070581030800010904010002034C
:1002A000000000092111010001222200070582033C
:1002B00020000107050303200001090402000103D7
:1002C00000000009211101000122B6000705840386
:1002D000200001120100020000000869EB05600126
:1002E00000010203011C037600690061006C003A02
:1002F00000660036003400630032006200330063A1
:100300000000000C0369006D006900360030000039
:10031000000E036B0065007900740065006E00003C
:10032000000403090429001E001F002000210022F0
:1003300000230024002500260027002D002E003178
:10034000002B0014001A000800150017001C0018EC
:10035000000C00120013002F0030002A00E00004FF
:10036000001600070009000A000B000D000E000F28
:10037000003300340028003500E10001001D001B9F
:100380000006001900050011001000360037003883
:1003900000E50021523900E3000000E20000000007
:1003A0000000002C00000000000000E600E700E470
:1003B0000001003A003B003C003D003E003F004091
:1003C00000410042004300440045000100390001A3
:1003D0000001000100007C0100010001000100019A
:1003E000004600520049004C000100AA00A900A8E4
:1003F0000001000100010001004B004A0050004FC5
:1004000000010001000100010001000100010001E4
:10041000000100010001004E004D005100010001EB
:1004200000010001000000010000000000000001C8
:1004300000000000000000010001000100FD377A0B
:10044000585A000004E6D6B4460200210116000006
:1004500000742FE5A3E0040701855D003D8889C68F
:100460005436C3174FE4F3730DE1698FFC64909B1E
:1004700036B1A3E2B9DE278383C8F46DCEF6AD169C
:1004800025FFEDA3224789BFC8DCC4CFDE23C537D3
:10049000EAAC0A37713C60D868C2AD48F9C5C5B549
:1004A000A1F23AAF4F31CCBA7AB93F55A41FEDB59E
:1004B000C62675667E4A7158144B2B9BAF2519686A
:1004C000DAB25825F9E69DBF7F343DB9821D5089C7
:1004D000B471F72E9A2673AE0E3BB89CD42BFCBE9B
:1004E0001994413C59AB68F43170DA907C26EEFFE8
:1004F0004B3604BF66AC1494362E3B4F4335F5CED5
:10050000D9BF67DB1D7DE1E353702D88C9B15AB3B4
:1005100095139B4E132128CFDC8F3C7DADA37F012B
:10052000111A54E4DE19C5D7B91DEDE2062D3F17A7
:10053000DC5FED9121D30DABE4A465E43ECE05A9CB
:10054000150AA6B2D17ECE2F50F763339EE1A11CCF
:10055000E6BF203E0445EF9C9D7C0AFA9A93F2BBCD
:10056000E7009690C34AF04FE1366DC6AA4BA33E12
:100570007D9BCAEC95F129549E9F66C8BD6EDABC7E
:10058000B4A8718E8D4749447B82087A3E4222DCB2
:1005900005AA1BC0E9D4D88686EBED33E401A97D1A
:1005A0001F380D817876356ADA22E45C41B7F3F9B9
:1005B000B99F8E203EA8AE41D60ABE5D4F2C61DAAF
:1005C0006959B113FA0C977473773C226B4BF4544E
:1005D000BED9B00FFF81AF8898D83AB2F8DEE4A553
:1005E0000000000000CF21C6DB34812C5A0001A19D
:1005F00003880800002AA34B70B1C467FB02000007
:10060000000004595A504F52514A4D4B4E2A4C2F1C
:1006100030B6B7ABACBBBCA9AABDBECFD0CDCEDB8C
:10062000DCD9DA0D0E0B0F1A05080509050718119C
:10063000130408120C0011241FBECFEFDAE0DEBF56
:10064000CDBF04B603FE18C080916005909161058E
:10065000A0916205B09163058730904BA740B04BE5
:1006600059F4109260051092610510926205109283
:100670006305E0E0F8E3099511E0A0E0B1E0E0E90E
:10068000F4E602C005900D92AA3AB107D9F725E029
:10069000AAEAB1E001C01D92A036B207E1F70E94BC
:1006A0001C280C94CA31ACCC9C019A9581159F41B1
:1006B00018F5F32FF270EE27832F8170732F74706B
:1006C0006627532F5870442734FF0CC08295807FD3
:1006D000EF2B09F08062672B09F08064452B69F0ED
:1006E00080680895EF2B09F08260672B09F0846021
:1006F000452B19F08860089580E00895CF93DF932B
:10070000EB01D2DFFE010995DF91CF9108950C94A2
:10071000EA300895982F92959F7024E0911102C0BD
:1007200020E0982F892F86958695811511F02E5FF0
:10073000982F892F8695820F089580935C050895E0
:1007400080935D05089521E030E001C0220F8A9575
:10075000EAF780915D05822BF3CF21E030E0A9011B
:1007600002C0440F551F8A95E2F7CA018095909107
:100770005D058923E5CF292F953090F58E3080F5E2
:1007800090E03EE0239F800D911D1124282F2770BB
:1007900041E001C0440F2A95EAF723E0969587953A
:1007A0002A95E1F7FC01EE0FFF1FE80FF91FEA5F42
:1007B000FC4F20E030E070E05191DF01CB01022ED0
:1007C00002C0969587950A94E2F7817081958527F6
:1007D000842385278E932F5F3F4F2330310561F7A8
:1007E0000895292F953078F58E3068F590E03EE039
:1007F000239F800D911D1124682F677023E096952B
:1008000087952A95E1F7FC01EE0FFF1FE80FF91F0E
:10081000EA5FFC4F40E050E080E0219130E0062E9E
:1008200002C0369527950A94E2F721703327042EEB
:1008300001C0220F0A94EAF7822B4F5F5F4F4330CB
:10084000510559F7089580E0089590915D0521E0E4
:1008500030E0F90101C0EE0F8A95EAF7D90102C034
:10086000AA0FBB1F6A95E2F7EA2B01C0220F4A9537
:10087000EAF7892F8E23E81303C0892F822B60CFDC
:100880002095822F8923FBCF8091B4029091B302EF
:10089000981301C008958F5F8770FACF9091A804D4
:1008A000809589238093A804282F2770211110C0D8
:1008B000891771F090915F0592FF0AC08695869521
:1008C00086954BDF1092A8041092AA041092A904F6
:1008D00008959091A504982B9093A5040895982FBE
:1008E00090958091A50489238093A5040895809113
:1008F000A404811531F01092A4041092AC0410925B
:10090000AB040895803E9105D9F1C8F48133910577
:1009100009F482C048F48932910509F472C08A3220
:10092000910509F480C0089589339105E9F0823872
:100930009105D1F08533910509F45EC00895843E98
:100940009105D9F148F4823E910539F1833E910534
:1009500049F181EE90E00895863E9105C9F1873E08
:10096000910509F43EC0089520915E052370211180
:1009700064C020915F0523FF14C089E290E00895D0
:1009800020915E0520FD45C030915F0530FF09C014
:1009900024FD24C083EE90E0089520915E0522FDA1
:1009A000F7CF089520915E0522FD44C030915F0588
:1009B00030FD43C024FFF5CF11C020915F0521FF1A
:1009C000F0CF80915E0584FD09C087EE90E0089528
:1009D00020915E0523FFE5CF24FFF7CF80E090E074
:1009E000089520915E0523FD2BC030915F0531FFF6
:1009F000E1CF84EE90E0089520915E0525FFD1CFF0
:100A0000BCCF20915E0525FD1EC020915F0523FF10
:100A1000C8CF89E390E0089520915E0526FFC1CFFD
:100A20008AE290E0089520915E0526FFBACF81E327
:100A300090E0089582EE90E0089580EE90E00895B1
:100A400086EE90E0089585E390E0089590915E052C
:100A500092FF10C041E0282F2471243009F040E0BB
:100A600031E0282F2871283009F030E0431711F0C9
:100A70002CE0822793FF10C041E0282F24712431FD
:100A800009F040E031E0282F2871283109F030E0EA
:100A9000431711F02CE0822730915F0530FF10C022
:100AA00051E0282F2171213009F050E041E0282F3A
:100AB0002871283009F040E0541711F029E082270E
:100AC00031FF10C041E0282F2171213109F040E0B1
:100AD00031E0282F2871283109F030E0431711F058
:100AE00029E0822794FD877E08951F93CF93DF939B
:100AF00009DFEC01811522E5920708F052C081154B
:100B000040E5940708F0CDC0803E910520F58D3C6E
:100B1000910508F0A1C0883A910570F4853A9105D5
:100B200008F097C081309105B9F10497813A910599
:100B300098F1C0E0D0E030C0885A91094B97C8F7CF
:100B4000C85AD0E0CC0FDD1FC35CDE4F0990D881BE
:100B5000C02DD46421C0811550E49507B0F4C115AF
:100B600080E2D80708F0B3C0C83ED105A8F0CE0196
:100B70009A9581159F41E8F68D2F68DF182FCE01D9
:100B80009927C0DEEC01D12B07C09927BBDECC270B
:100B9000DF70C82BD92BD06ACE01DF91CF911F9186
:100BA0000895803842E59407C8F5803652E59507E8
:100BB00008F05BC0C03482E5D807D0F4C03292E5BB
:100BC000D90708F04BC08C2F8695869520E2829F2E
:100BD000C0011124C37021E030E0A90102C0440F1C
:100BE000551FCA95E2F7EA01C82BD92BDD68D4CF8F
:100BF0008C2F86958695877050E2859FC0011124C1
:100C0000C37021E030E0A90102C0440F551FCA950E
:100C1000E2F7EA01C82BD92BDC68BECF803C52E555
:100C2000950758F48F71C03AD245A0F590E0982FFF
:100C30008827EC01C46FD06AAFCF805C9245809763
:100C400008F077CFDC2FCC27CC27DF71C06FD06ABC
:100C5000A3CFA497D064A0CFD0659ECFCF71D0E0B2
:100C6000DC2FCC27C16FD06A97CF86958695877089
:100C700020E2829FC0011124C37021E030E0A9016D
:100C800002C0440F551FCA95E2F7EA01C82BD92BC1
:100C9000DA6882CFDBDEC82FD0E0DC2FCC27D06231
:100CA0007BCF8F71D3DE93E0CC0FDD1F9A95E1F7F8
:100CB000CC27DF70282F30E084FF05C050E1859FEE
:100CC000900111243327C22BD32BD06965CF8D2FF0
:100CD0008F71BCDE182FCE01992714DEEC01D12BC9
:100CE000DECF80E00895F894E82FE295EF70F0E011
:100CF00041A18F7021E030E0B90102C0660F771F7B
:100D00008A95E2F7CB01962F9095942391A392A117
:100D1000892B82A37894089581152CE7920741F4DA
:100D20002091800230918102232B11F480E090E029
:100D30000895EDE1F4E080E090E06AE876E24DEAC3
:100D400056E22FE137E27783668351874087338706
:100D5000228797878687019670968830910599F744
:100D60000895FB01811520E2920728F4811541E0E6
:100D7000940738F408959C0130522115304348F00F
:100D80000895392F94FF02C03295307F2081232BA4
:100D9000208399270895462B22FF0FC0982F929504
:100DA0009F708F70892B962F92959F706F70692B13
:100DB000942F92959F704F70492B982F96239613DE
:100DC00009C050E04095509590E04823592381E0B8
:100DD000452B09F080E008951092EE041092ED0486
:100DE000EDEAF4E08581811102C014821682379603
:100DF00084E0E53EF807B1F70895AC013091F004C6
:100E00006091EF04232F621301C00895822F90E0B8
:100E1000FC01EE0FFF1FEB51FB4F0190F081E02D25
:100E2000E417F50791F467E0649FF001659FF00D0A
:100E30001124E355FB4F41E044832313E6CF019691
:100E4000837099278093F00408950196282F2370CA
:100E5000DACFFC018481862381110AC08281811549
:100E6000B9F06823908593FF05C081E061110FC040
:100E700080E00895282F22952F708F70282B962FB1
:100E800092959F706F70962B81E02913F1CF089592
:100E900081E008950F931F93CF9301E010E0082E97
:100EA00001C0000F0A94EAF7C091A3049C2F90237D
:100EB000911115C09091A8049695969596958913D1
:100EC00006C01092A8041092AA041092A9043BDC58
:100ED000C027C093A304CF911F910F9108953DDCCB
:100EE000F7CF282F35EB2303C001112497FF04C04F
:100EF00080589109892F089580589F4FFBCF80918A
:100F0000230380FD14C081FD14C082FD16C08091B2
:100F10002203811581F08E3180F420E5829FC0018B
:100F200011246EE170E00E94D130862F089584E193
:100F3000089588E2089588E0089580E508958091F5
:100F4000230380FD17C081FD17C082FD19C0809169
:100F50002103811599F0883298F428E0829FC0011E
:100F6000112468E270E00E94D1306115710551F0E2
:100F7000862F089562E0FCCF64E0FACF61E0F8CFFD
:100F800068E0F6CF81E0089590917F038902900197
:100F9000112437FF03C080937F0308952F37310555
:100FA0001CF4980F90937F0308959C0180E090E0DB
:100FB000F901E80FF91FE491E41307C091E08927D4
:100FC000F901E80FF11D849108950196861780F3C9
:100FD00080E00895FA01309709F009950895E091AD
:100FE000A902F091AA02309739F00190F081E02D2A
:100FF000309711F00995089580E00895A3E0B0E0DE
:10100000E4E0F8E00C9411319C018091F2019091A0
:10101000F30182179307B1F03093F3012093F201AB
:10102000E091A902F091AA02309761F00084F18565
:10103000E02D309739F083E089833B832A83CE010A
:10104000019609952396E2E00C942D31A3E0B0E0DF
:10105000ECE2F8E00C9411319C018091F001909148
:10106000F10182179307B1F03093F1012093F00161
:10107000E091A902F091AA02309761F00084F18515
:10108000E02D309739F084E089833B832A83CE01B9
:10109000019609952396E2E00C942D3190910E0172
:1010A000913091F0AEEAB1E0EFEF90E02D91821730
:1010B00051F0EF3F19F4211101C0E92F9F5F9630E5
:1010C000A9F7EF3FC9F4089590915E0597FFEACF25
:1010D000E82FE695E695E695803FA8F7F0E0EC541A
:1010E000FE4F877021E030E001C0220F8A95EAF7B9
:1010F0008281822B828308950E2E000CFF0BE45513
:10110000FE4FF8CF90910E01913021F490915E0541
:1011100097FD0CC0EEEAF1E09191891302C0DF0166
:101120001E9251E0E43BF507B9F70895E82FE695E4
:10113000E695E695803FC8F7F0E0EC54FE4F8770E7
:1011400021E030E0A90102C0440F551F8A95E2F763
:10115000CA018095928189238283089580910D012F
:1011600008952FB7F8948091EC019091ED01A09132
:10117000EE01B091EF012FBF0895CF93DF93C0919F
:10118000A5048091A704C82B8091A4048115F1F0D7
:10119000E8DF2091AB043091AC04821B930B8838BC
:1011A000934108F0A4DBD091A40480910E0181301A
:1011B00021F480915E0587FD13C086E02EEA31E0C0
:1011C00090E0815088F4911192DBCD2B80919903AE
:1011D00080958C2390919803892BDF91CF9108956E
:1011E0008EE126EB31E0ECCFF90141919F014115F1
:1011F00041F39F5FE6CF962F20915F0522FF0EC03F
:10120000682F660F660F660F692B6093A8049BDA40
:10121000A8DF9093AA048093A904089594CA90919A
:10122000A404292F2823211559F080958923809320
:10123000A404811531F095DF8093AB049093AC0446
:10124000089580E090E0F8CF8CDF20912603309164
:101250002703232B211521F080936F0290937002B6
:101260002091280330912903232B211521F080930D
:101270006D0290936E02E091A902F091AA0230975C
:1012800059F00680F781E02D309731F082E08093AD
:10129000240384E293E009950895611509F441C09F
:1012A000E3E3E80FE33148F4F0E0E453FE4C0C9440
:1012B000E43025DE819580932703C6CF20DEFBCF67
:1012C0001EDE819580932603F8CF19DEFBCF37DE33
:1012D00080932803F2CF33DE8195FACF30DE8195FB
:1012E00080932903EACF2BDEFBCF815D990B21E0B0
:1012F00030E001C0220F8A95EAF780912503822B06
:1013000080932503DACF80912303816080932303A8
:10131000D4CF809123038260F9CF8091230384602E
:10132000F5CF409126038D3C59F48091270387FF28
:101330000DC010922703411559F41092220308C0E2
:101340008E3C81F48091270318169CF3411581F09F
:101350008091280390912903892B8111AECF10929F
:101360002103ABCF8F3C41F447FFF0CF109226030F
:10137000809127038115E0CF803D19F41416B4F352
:10138000E5CF90912803893D29F41916FCF61092B7
:101390002803DCCF8A3D19F497FFD8CFF8CF90917E
:1013A00029038B3D29F497FFD1CF10922903CECF8B
:1013B0008C3D19F41916CCF3C9CF9FE2980F9830E1
:1013C00090F4815D990B21E030E0B90102C0660F15
:1013D000771F8A95E2F7CB018095909125038923A9
:1013E00080932503B3CF8D3D31F4809123038E7F0D
:1013F00080932303ABCF8E3D21F4809123038D7F17
:10140000F7CF8F3D09F0A2CF809123038B7FF0CFE0
:101410002FB7F8946091EC017091ED018091EE018D
:101420009091EF012FBF0895CF92DF92EF92FF923C
:10143000CF93DF93D82FC92FC0901704D0901804F2
:10144000E0901904F0901A04E3DF6C197D098E090D
:101450009F09643F71408105910510F1D9DF6B014F
:101460007C0182E390E0A0E0B0E0C0926902D092FB
:101470006A02E0926B02F0926C0280936502909394
:101480006602A0936702B0936802D0931504C093DC
:101490001604DF91CF91FF90EF90DF90CF900895E9
:1014A00084EF91E0A0E0B0E0E0CFFC019B018091EF
:1014B000E2019091E3018617970740F0672B29F42A
:1014C0008091E8008E778093E800C90140E00097A2
:1014D00041F4411106C08091E80082FF2FC080E0F6
:1014E0000895209182022115A9F12530A9F12091BA
:1014F000E80023FD2DC02091E80022FDECCF2091D3
:10150000E80020FFE4CF3091F3002091F200009733
:1015100019F02830310558F041E02830310509F044
:1015200040E02091E8002E772093E800D0CF419151
:101530004093F10001972F5F3F4FE9CF80918202E6
:10154000811541F0853041F08091E80083FFC3CFE1
:1015500081E0089582E0089583E008958091DC01A0
:1015600087FF13C08091E80082FF06C08091E800E9
:101570008B778093E8000895809182028111F2CFE9
:101580000895809182028115D9F38091E80080FF4F
:10159000F8CF8091E8008E77ECCF2091E400309175
:1015A000E50095E6A9012091EC00822F817020FFD3
:1015B00006C08091E80080FF06C080E00895209179
:1015C000E80022FD1AC080918202811589F08530E1
:1015D00089F08091EB0085FD0FC02091E4003091EF
:1015E000E50042175307F9F29A95E1F684E0089571
:1015F00082E0089583E0089581E00895E8EDF0E049
:1016000080818E7F80831092E2001092DA00109227
:10161000E100A0EEB0E08C9181608C9380818F77A7
:10162000808319BCA7EDB0E08C918E7F8C93808174
:101630008F7E80831092DB010895E091A902F091E2
:10164000AA02309739F00284F385E02D309711F02B
:1016500060E209950895982F9093E900891771F039
:101660007091EC002091ED005091F00021FD09C037
:101670009F5F973089F78093E9000895762F242F94
:1016800050E03091EB003E7F3093EB003091ED0065
:101690003D7F3093ED003091EB0031603093EB00F3
:1016A0007093EC002093ED005093F0002091EE0039
:1016B00027FDDECF0895A0E0B0E0E1E6FBE00C946A
:1016C0000B31C8EDD0E088818F7E8883E7EDF0E0B4
:1016D00080818160808384E082BF81E08093DB0130
:1016E00088818E7F888302EE10E0F80110821092CC
:1016F000DA0081EEC82ED12CF601108288818F7716
:10170000888388818068888388818F7D888319BCDD
:10171000109282021092DA01109259021092D901AD
:1017200090EEE92EF12CF70180818B7F80838881F8
:101730008160888342E060E080E08DDFF601808197
:101740008E7F8083F80180818160808380818860C2
:101750008083F70180818E7F808388818061888388
:10176000CDB7DEB7E8E00C942731E091B402909158
:10177000B30229E0E91302C080E00895AE2FB0E083
:101780002E9FF0011124EB54FD4F3181361306C01A
:101790003081381303C03581341304C0FD01319604
:1017A000E770E8CF81E0089581E08093E00080E277
:1017B0008093D8001092C9008FE19EE40197F1F761
:1017C00000C0000087E090EBDC01809360059093FF
:1017D0006105A0936205B093630588E19CE00FB6B4
:1017E000F894A895809360000FBE90936000FFCF9F
:1017F0000F931F93CF93DF938B01EA0190918202A5
:10180000943051F58093E9008FEF9091E80095FDB9
:1018100006C095ED9A95F1F700008A95B1F7809191
:10182000E80085FF19C0B9DE811111C08091E80080
:1018300085FD06C08091E8008E778093E800F3CFA5
:10184000F80181918F018093F100219779F78091C0
:10185000E8008E778093E800DF91CF911F910F9180
:101860000895792F603229F440E250E0682F82E039
:10187000BFCF0895CF93DF93D82FC92F48E050E012
:10188000682F792F81E0B4DF88E0ED2FFC2FA4EEE4
:10189000B1E001900D928A95E1F7DF91CF91089523
:1018A000BC0140E250E084E0A3CFBC0146E050E040
:1018B00084E09ECFBC0143E050E084E099CF90915A
:1018C0005F0592FB222720F9281779F080FB92F917
:1018D00090935F0560915E0570915F0584E090E0F4
:1018E0000E94AF3182E00C944E0408951F93CF9371
:1018F000DF93962F122F632F8430D8F49530C8F4DD
:101900004E30B8F4C42FD0E0CC0FDD1F2CE1929FF5
:10191000C00DD11D11249CE8899FC00DD11D11243B
:10192000CE0189960E949531612FCE018A960E9440
:101930009531DF91CF911F91089580910E018130F3
:1019400061F580915E0587FF28C017DC8093B501A3
:1019500040E250E069E872E084EB91E00E9455318A
:10196000892BD1F080E2E4EBF1E0A9E8B2E001904C
:101970000D928A95E1F7E091A902F091AA023097C1
:1019800059F00480F581E02D309731F086E08093A6
:10199000B40184EB91E009950895EFDB8093AC01ED
:1019A00048E050E06BEA72E08CEA91E00E94553129
:1019B000892B91F388E0ECEAF1E0ABEAB2E0019028
:1019C0000D928A95E1F7E091A902F091AA02309771
:1019D00019F30280F381E02D3097F1F28CEA91E067
:1019E000DACF811519F00E946904A7CF08958115F7
:1019F00031F09091A704892B8093A7049ECF08957E
:101A0000CF93C82F8115C1F08CEF8C0F813A80F5F0
:101A100080910E01813021F480915E0587FD0EC01A
:101A2000EEEAF1E08191C817F9F021E0E43BF2071A
:101A3000C9F78C2F33DB81DFCF910895EC2FE6952A
:101A4000E695E695F0E0EC54FE4F828190E04C2F55
:101A5000477021E030E002C0220F331F4A95E2F7C1
:101A600082239323892B29F38C2F4CDB66DFE1CF74
:101A700080E28C0F883048F4C77081E001C0880F85
:101A8000CA95EAF70E946904D6CF8BE58C0F8330A4
:101A900030F42C2F2452330BC901B0DACDCFE8E556
:101AA000EC0FEB3148F4F0E0EE0FFF1FED58FE4F66
:101AB00080819181CBDAC0CF83E38C0F833108F032
:101AC000BBCF61E08C2FE9DBB7CFCF93DF93EC0185
:101AD000805E9109089720F067EF7CE0209711F471
:101AE00061EF7CE0CE010E947E038C2F89DFDF91C5
:101AF000CF910895811541F19CEF980F913A10F420
:101B000001DB1BCF90E2980F983050F4877091E082
:101B100001C0990F8A95EAF7892F0E946F04F1CFCF
:101B20009BE5980F933018F480E090E067CA98E541
:101B3000980F9B3118F480E090E088CA93E3980FE7
:101B4000933110F460E0A9CB08951F93CF93DF93F6
:101B5000182FEB0155DF209731F4812FCBDFDF9178
:101B6000CF911F9108958FE99FE00197F1F700C091
:101B700000002197F0CF811519F00E946F04DDCE8F
:101B80000895811539F080959091A7048923809359
:101B9000A704D3CE089580919403811521F082E2A9
:101BA000F0DF1092940308951092A50480910E0125
:101BB000813011F580915E0587FF1EC0E6EBF1E0F4
:101BC0008EE1DF011D928A95E9F780E090E016DA58
:101BD00080E090E03BDA1092A704AFDE86E0E4E21A
:101BE000F3E0DF011D928A95E9F71092220310922B
:101BF00021031092230328CBEEEAF1E086E0E1CF47
:101C0000D3DF2FEF84E39CE0215080409040E1F748
:101C100000C0000088E19CE00FB6F894A89580937E
:101C200060000FBE90936000FFCFAAE2B0E0EBE14E
:101C3000FEE00C9410318CED91E0FC0101962091B6
:101C4000F100208321E0843E9207B9F78091DD0105
:101C5000893009F457C0C8F4823009F4B2C0833027
:101C600009F482C0813081F18091E80083FFE6C0F1
:101C70008091DC019091DD019A3008F0DFC0E92FFE
:101C8000F0E0E152FE4C0C94E4308A3009F489C053
:101C90008B3051F78091DC01813231F78091E00186
:101CA0009091E101892B01F78091E800877F809373
:101CB000E80054DC81E09091DE01911101C080E0E8
:101CC00080930E0171DFD0CF8091DC01813A61F603
:101CD0008091E800877F8093E8008091E0019091F7
:101CE000E101892B59F060E080E090E070E0DDDBFD
:101CF0008091E8008B778093E800B6CF68E084EEAF
:101D000091E0F4CF8091DC01813209F0ADCF809178
:101D1000E0019091E1018D7F892B09F0A5CF8091A1
:101D2000E800877F8093E8008091E80082FF17C079
:101D30009091F3008091F200029731F48091F100CC
:101D4000813011F0863021F48091F10080930D01F3
:101D50008091E8008B778093E80000DC85CF80914C
:101D600082028111E1CF80CF8091DC01813A09F0BC
:101D70007BCF8091E0019091E101892B09F074CF34
:101D80008091E800877F8093E8008091E80080FFE1
:101D9000FCCF80910E018093F1008091E8008E7756
:101DA000DACF8091DC01813209F05ECF8091E800CA
:101DB000877F8093E800D2DB8091DF0180930C0164
:101DC00053CF8091DC01813A09F04ECF8091E80039
:101DD000877F8093E8008091E80080FFFCCF8091AE
:101DE0000C01D9CF803889F0823841F58091E0012B
:101DF0008F70873018F58093E9008091EB0085FBA8
:101E0000882780F91092E90006C080915902880F56
:101E10009091D901892B9091E800977F9093E800E9
:101E20008093F1001092F1008091E8008E7723C03A
:101E3000811116C08091DE01813009F18091E800A6
:101E400083FF0AC08091E800877F8093E80080913B
:101E5000EB0080628093EB00AA96E3E00C942C31B7
:101E6000823061F78091DE01811581F01092E900E6
:101E70008091E800877F8093E80070DBDFCF81E00E
:101E8000933009F080E080935902F0CF8091E00117
:101E90008F702FEF280F263088F68093E90020916D
:101EA000EB0020FFE3CF933031F48091EB008062B0
:101EB0008093EB00DBCF9091EB0090619093EB006F
:101EC00021E030E0A90102C0440F551F8A95E2F7D6
:101ED0004093EA001092EA008091EB008860E8CF1E
:101EE0008111ACCF1091DE011F778091E3008078E3
:101EF000812B8093E3008091E800877F8093E80046
:101F00002DDB8091E80080FFFCCF8091E3008068AA
:101F10008093E30083E0111101C082E0809382028C
:101F20008DCF8058823008F089CF8091DE0190916A
:101F3000DF018C3D53E0950791F583E08A838AE2C7
:101F400089834FB7F894DE01139620E03EE051E21A
:101F5000E32FF0E050935700849120FF03C0829557
:101F60008F703F5F8F708A30C0F0895C90E08D93F6
:101F70009D932F5F243161F74FBF8091E800877FE9
:101F80008093E8006AE270E0CE0101968EDA8091DB
:101F9000E8008B778093E80051CF805DE7CF292F51
:101FA00033272330310509F44EC078F5213031054F
:101FB00009F488C08BE590E0E8E7F2E022303105D3
:101FC00009F03CCF2091E800277F2093E800209182
:101FD000E2013091E3018217930708F49C0140E08D
:101FE0002115310509F073C0411171C08091E800DD
:101FF00082FDCDCF80918202811549F2853039F280
:102000008091E80083FFF2CFC2CF8091E0019091F0
:10201000E1012132310509F446C02232310509F0CF
:102020000DCF8330910508F009CFFC01EE0FFF1FA3
:10203000E25EFE4F0190F081E02D855E9E4FDC0157
:102040008C9190E010C09C013327823021F1233025
:10205000310568F4232BB9F4E1E2F3E0E4918E2F2B
:1020600090E0E1E2F3E0009709F4E8CEABCF233053
:10207000310509F0E3CEE5EEF2E0E4918E2F90E039
:10208000E5EEF2E0F0CFE1E1F3E0E4918E2F90E0B5
:10209000E1E1F3E0E8CFE3E0F3E0E4918E2F90E0BC
:1020A000E3E0F3E0E0CF8330910508F0C7CEFC0118
:1020B000EE0FFF1FEC5DFE4F0190F081E02D89E0F7
:1020C00090E080CF82E190E0E3EDF2E07BCF809181
:1020D0008202811509F45BCF853009F458CF8091D5
:1020E000E80083FD54CF8091E80082FD7FCF80918E
:1020F000E80080FF75CF9091F3008091F2002115E8
:10210000310519F08830910550F041E0089709F049
:1021100040E08091E8008E778093E80061CF4491A1
:102120004093F1003196215031090196E8CF803873
:1021300009F084CE8091E800877F8093E800809149
:10214000DA018093F10070CE811178CE1091DE011A
:10215000123008F073CE8091E800877F8093E8000A
:102160001093DA01FBD91115D9F084E08093820233
:1021700042E061EC81E06FDA42E261EC84E06BDA2C
:1021800042E261EC82E067DA42E260EC83E063DA2B
:1021900080918202843051F482E080930F014ECE10
:1021A0008091E30087FDE1CF81E0E0CF81E0F5CFD2
:1021B000CF93DF93EC014A855B856E857F850E9416
:1021C000EA079B8190958091A70489238093A704B7
:1021D0008C810E946F04B1DB86E0FE0111928A952A
:1021E000E9F7DF91CF910895CF93DF93EC018D81D3
:1021F00081FD13C082608D838091A7049B81892B10
:102200008093A7048C810E94690497DB48855985D7
:102210006E857F85CE010E94EA0710929E0410927F
:102220009D048D8180FD02C0CE01C2DFDF91CF9180
:1022300008951F93CF93DF93182FA0911304B091AB
:102240001404109709F448C0109216041092150453
:1022500010929903109298031696CD91DC911797DE
:10226000CE019A9581159F4108F4D07ED1E0C1112D
:1022700001C0D0E01996ED91FC911A97309731F09A
:102280001B966D917C9180E00995D823D11539F08A
:102290008CEF8C0F813A20F58C2F0E94820811154B
:1022A000A1F0E0911304F0911404808584FD0DC029
:1022B00080911204811549F0808191819C01215007
:1022C00031092F333E4708F4AFD837DB109214049E
:1022D0001092130410921204DF91CF911F91089570
:1022E0002CDB8C2F07DCDBCF0F931F93CF93DF9377
:1022F000843030F5653020F54E3010F5C42FD0E035
:10230000CC0FDD1F2CE1629FC00DD11D11243CE8D4
:10231000839FC00DD11D1124CE0189960E94793171
:10232000082F10E0102F0027CE018A960E947931E5
:102330009801282BC901DF91CF911F910F9108952A
:1023400080E090E0F8CF462F672F209185023091F2
:102350008602232B81F4703F39F4403F61F4809171
:102360008302909184020895753028F44E3018F459
:10237000843008F4B9CF80E090E00895A0E0B0E0A8
:10238000E4ECF1E10C940C317C0100915D0580914D
:102390005C05082BC3E0D0E010E0C8010C2E02C0A1
:1023A000959587950A94E2F780FD09C02197A8F7D3
:1023B000D12C8D2DCDB7DEB7E7E00C942831DC2E83
:1023C000B7018C2FC0DF0E947505019779F3F1CF1B
:1023D0000F931F93CF93FC0187819085009789F419
:1023E000858100811181811581F0611571F0C8012D
:1023F000C5DFC82F682FC8010E94BB03B8018C2F0E
:10240000A2DFCF911F910F910895C8010E94F1039F
:10241000C82FF4CFCF93DF93D82FC92FAFDF6D2F05
:102420007C2F91DF0E947505DF91CF910895FC010B
:1024300084818115B1F0878190850097A1F00E9479
:102440007505282F92959F709630B9F080F4925FB1
:102450009F70923030F4203FD1F058F481E0283E54
:1024600058F080E0089580819181D4DFEACF9A5FAF
:10247000EFCF81E0243FA9F7089591E0813F09F073
:1024800090E081E0283E08F080E0892B089581E00B
:102490000895382F292FCB01A32FB22F873891050C
:1024A000A105B10520F487589C4F0C94793180E048
:1024B000089585E290E00E947931823F89F486E2B6
:1024C00090E00E947931823A59F487E290E00E94CC
:1024D000793191E0853509F090E0892F8170089578
:1024E00080E0FCCFAAE0B0E0E8E7F2E10C9406312E
:1024F000C0908002D090810281E090E090938102B0
:1025000080938002812C912C10E0540100E019C0CE
:1025100021E030E0123020F4F701859195919C0183
:10252000472D602F812FE2D9739422E0E20EF11C37
:102530003EE07312EDCF0F5F8EE0A80EB11C0530A8
:1025400049F0C501880F991FFC01EB5DFC4F7F012D
:10255000712CDECF1F5FF6E48F0E911C1430A9F6AC
:102560001A8219821C821B821E821D8218861F827B
:1025700088EC90E09A87898709E512E09E012F5F39
:102580003F4F79014AE050E0B801C7010E94B331E2
:10259000065F1F4F093A32E01307A1F78AE0F701FF
:1025A00011928A95E9F74AE050E0B801C7010E940C
:1025B000B331065F1F4F093FF2E01F07A1F789E023
:1025C000F70111928A95E9F78FEF9FEF9E838D8334
:1025D00087E08A874AE050E0B801C7010E94B33122
:1025E000065F1F4F0934F3E01F07A1F786E0F701EC
:1025F00011928A95E9F746E050E0B801C7010E94C0
:10260000B3310A5F1F4F0937F3E01F07A1F7D092DC
:102610008102C09280022A96EDE00C942231AAE059
:10262000B0E0E5E1F3E10C940B31E6EFF1E080E599
:10263000DF011D928A95E9F7EDEAF4E088E3DF0116
:102640001D928A95E9F786EFC82E81E0D82E7F018A
:1026500009EA12E0F701D182C0824AE050E0B801F5
:10266000CE0101960E94693188E0FE013196D601C3
:1026700001900D928A95E1F789859A85D701139685
:102680009C938E931297BAE0CB0ED11CE7E0EE0E2E
:10269000F11C065F1F4F093FF2E01F07D9F62A968B
:1026A000E8E00C942731AAE0B0E0E9E5F3E10C940E
:1026B00009310AE913E089EFE82E82E0F82E97E06D
:1026C000B92E25EFC22E21E0D22EAA24A3944AE0EF
:1026D00050E0B701CE0101960E946931F8013896A9
:1026E000DF018B2D1D928A95E9F789819A81D801A6
:1026F00011969C938E938F8112968C9312978D8155
:1027000013968C931397888514968C9314978985C8
:1027100015968C9315978B819C8117969C938E931D
:1027200016978A8587FD04C01E96DC92CE921D976F
:1027300080FF02C0F801A08681FF07C0D80118966B
:102740009C911897926018969C9382FF04C0F801A0
:1027500090859460908783FF07C0D80118969C915C
:102760001897986018969C9384FF04C0F801908590
:102770009061908785FF07C0D80118968C911897B3
:10278000806218968C93BAE0EB0EF11C015F1F4F2C
:10279000E9E4EE16E3E0FE0609F099CF2A96EAE0B6
:1027A0000C942531A6E0B0E0E8EDF3E10C940C3197
:1027B00004E313E089E4E82E83E0F82E98E0D92EB4
:1027C00046E050E0B701CE0101960E946931F80160
:1027D0008D2D11928A95E9F7B8016C5F7F4F898141
:1027E0009A810E94B106F80191838083B8016B5FE2
:1027F0007F4F8B819C810E94B106F8019383828375
:102800008D8186838E818783F6E0EF0EF11C085F51
:102810001F4F89E7E81683E0F80691F62696E7E071
:102820000C942831282FCB01283070F44AE0249FE3
:1028300090011124B901675A7D4F4AE050E00E948F
:10284000693180E090E008958FEF9FEF0895AAE04E
:10285000B0E0EDE2F4E10C9411319C019755811543
:10286000914068F4BE016F5F7F4F822FDBDF892BC1
:1028700031F489859A852A96E2E00C942D3188EC12
:1028800090E0F9CFA0E0B0E0E8E4F4E10C940C3182
:10289000162FD72FC42FD22E8115A1F04093A1045B
:1028A0000E94B1089093D8018093D701C77081E04E
:1028B00001C0880FCA95EAF794D8CDB7DEB7E7E034
:1028C0000C9428319091A104491335C0E090D701B0
:1028D000F090D8010E94B1089C012E193F0979019E
:1028E000812F9D2FB4DFE816F90628F5D0E2DD0D23
:1028F000CD1591F0C77011E0812F01C0880FCA95E6
:10290000EAF739D9D83040F48D2D877001C0110F06
:102910008A95EAF7812F65D860E070E0802F15D99D
:10292000D83058F62D2D277081E001C0880F2A95E8
:10293000EAF721D9C2CFC77081E001C0880FCA95DC
:10294000EAF7F7CFA0E1B0E0E8EAF4E10C94033154
:10295000FE01319680E1DF011D928A95E9F709E0D9
:1029600010E099E7A92E93E0B92E27E8422E512CCA
:10297000612C712C4F0173016201B1E14B165104BE
:10298000610471041CF080E1C82ED12CA601B501B0
:10299000C4010E948631AC0CBD1C0D2C000CEE084D
:1029A000FF084C185D086E087F080150104019F7A9
:1029B0006096E0E10C941F316FEF85E290E00E9499
:1029C00095316FEF86E290E00E9495316FEF87E2DC
:1029D00090E00E94953160E088E290E00E9495319D
:1029E00081DDB0DF62EF85E290E00E94953162EA1E
:1029F00086E290E00E94953165E587E290E00C94D4
:102A00009531A0E0B0E0E7E0F5E10C940A31EC018B
:102A10008881811511F1813009F046C089818130AA
:102A200051F48A81239660E570E0893311F060E00B
:102A300070E08BD8EDCF823029F48A8123960E94F2
:102A4000000DE6CF833021F48A81239653D8E0CF5E
:102A5000843041F022968111DBCFCDB7DEB7E9E0BB
:102A60000C9426318A81239620E030E09AE0682F8A
:102A70006053770BAB016A30710560F021153105A9
:102A800051F3EFE9FFE03197F1F700C0000021506A
:102A90003109F4CF929FB001939F700D11249A01D8
:102AA000260F371F8991E3CFE82FF0E0E850FE4F63
:102AB000B490282F26952695269530E0F901E85107
:102AC000FE4FE4908770F12C082E02C0F594E79435
:102AD0000A94E2F7E0FAEE24FF24E0F8F901E85264
:102AE000FE4FC490D12C082E02C0D594C7940A94EE
:102AF000E2F7C0FACC24DD24C0F8F901E853FE4F18
:102B0000049110E002C0159507958A95E2F70170CF
:102B10001127E114F10419F081EE0E94000DC11497
:102B2000D10419F086EE0E94000D60E070E08B2D5C
:102B30000CD8C114D10419F086EE0E947A0DE1146C
:102B4000F10419F081EE0E947A0D0115110529F0AA
:102B500060E070E08CE20E94A50D219659CFACE0B8
:102B6000B0E0E5EBF5E10C9401317C01DC01149659
:102B70008C91811509F44AC161E0C70129DC8C01FF
:102B8000F7018581811521F180919D0490919E042A
:102B90000097F1F008171907D9F0FC01FF27887F8B
:102BA0009927892B09F04BC0B4E0EE0FFF1FBA95AF
:102BB000E1F7E35EFB4F85818460858311830083A9
:102BC000CF0112DB1092A70461E0C70101DC8C0188
:102BD0008091890381113AC0D70115968C91811596
:102BE00009F4C9C00115B0E51B0708F0AFC0011515
:102BF000E0E21E0708F00EC10115F7E01F0731F1F2
:102C000008F5C801805E9109089700F13091A5048C
:102C10008091A7042091A40499E0F701A5E7B3E00F
:102C200001900D929A95E1F710937D0300937C0338
:102C300010927F03832B822B8093740307C0E0E004
:102C4000F0E0B9CF01153FE0130701F7F7018581E7
:102C50008111DDC1011527E5120708F4E6C201154F
:102C600038E5130710F00C945C20680147E5D41A8E
:102C70006AE873E08C2DD6DD892B31F5C601E4E0DE
:102C8000880F991FEA95E1F7FC01E35EFB4F228173
:102C9000213009F09AC220918A0330918B03232BB3
:102CA00099F020918C0330918D03232B69F02091B2
:102CB0008E0330918F034091900350919103242B08
:102CC000352B232B09F48BC280919403811509F4D1
:102CD00030C3C090A504D090A4040E94B1088857C6
:102CE0009C4E9093960380939503D70115968C91F3
:102CF000811509F41EC38D2D8C298D7981114CC34A
:102D00000115B0E51B0708F0E6C20115E0E41E0757
:102D100008F049C3063E110509F40BC3C8019052DF
:102D20008115904208F046C3D70116968C918031E8
:102D300008F42AC3C80199271092A7048D3291057F
:102D400009F0E2C282E08093A70438C3003E42E566
:102D5000140750F4003652E5150708F077CFC80184
:102D600092558034910551CF980127573C47253023
:102D7000310508F04BCF0937BCE71B0709F04FC0FE
:102D800020917C0330917D03232B79F18115A1F0F3
:102D900081E00E94C407809174030E94F70C89E0CF
:102DA000E5E7F3E0ABE2B3E001900D928A95E1F73D
:102DB00080917F0380932A0386E0F701ABE2B3E0C2
:102DC00001900D928A95E1F780912A0380938903FF
:102DD0008BE293E0C4DE10928903F70185818111B3
:102DE00004C0809174030E94C10D8091A804877073
:102DF000811561F0D70115968C91811539F080917C
:102E00005F0582FF03C082E00E944E042C96E2E13F
:102E10000C941D31D70116968C918031F6CE0A376D
:102E2000FCE71F0709F012CF811509F4C5C0A09077
:102E30007C03B0907D03209174032D832983BE0110
:102E40006F5F7F4FC5010E94B1062C0139813B871E
:102E5000A4E3CA2EA3E0DA2E01E010E022242A9493
:102E6000D60117963C90179733FE53C06D907C9017
:102E7000119712968D909C90139746145704B9F4AD
:102E80001496BC91B987232DF60146816B2F8B8553
:102E90000E94CB06811559F089850E948703281668
:102EA00034F4D60115969C918401192B282E4814D0
:102EB0005904C9F431FE17C0F601F581F987232DB5
:102EC000D60116964C916F2F8B850E94CB068115EB
:102ED00051F089850E94870328162CF4F60194810D
:102EE0008301192B282E30FE14C0FFEF2F1211C0C2
:102EF0000130110571F4232DD60116964C9160E036
:102F00008B850E94CB06811521F0F6018581840115
:102F1000182BF8E0CF0ED11C24E733E02C153D052B
:102F200009F09ECF01301105E1F58D8182958F70FA
:102F30003D81832B8F7011E0303108F410E0129541
:102F4000107F182BA11440E2B40620F5A11451E023
:102F5000B50608F055C00A2D812F8D704A2D8115B8
:102F600009F451C06AE08BE296E00E94D507282F51
:102F700030E02115310551F4402F6EE185E096E0F7
:102F80000E94D507282F30E0811549F0F901F12B77
:102F90008F0107C0C50190528115904390F100E068
:102FA00010E087E0E0E8F3E0DF011D928A95E9F7A1
:102FB000109388030093870380918703909188037F
:102FC000892B09F412CFF7018581811539F08FEF34
:102FD0000E94C40780917F0380937E0386E0F701FF
:102FE000A0E8B3E001900D928A95E1F780917E030D
:102FF0008093890380E893E0B2DD10928903F5CED7
:103000001B29BB24A8CF68E083E296E0AECFC801BD
:1030100097578038910508F0EDC0003108F0E5CEF3
:1030200066E870E080E090E034DA8111DECE812C39
:10303000912C5401011143C004E0AE014F5F5F4F7A
:103040006A01D601E02F1D92EA95E9F724013501C6
:10305000FFEF4F1A5F0A6F0A7F0AC501B40119DA40
:103060008983811509F4C1CE813009F0ABC0A50177
:1030700094012E5F3F4F4F4F5F4F2D833E834F8311
:103080005887C301B20105DA182F8A83811509F424
:10309000ACCE8FEF810F833050F56D817E818F81B3
:1030A0009885F7D98B83811511F0C601AADC24011C
:1030B000350133E0430E511C611C711C46C0F7E81A
:1030C0008F169104A104B10409F48FCEC501B40197
:1030D000E0D92FEF821A920AA20AB20A8111EFCF29
:1030E0000150A8CF4D805E806F8078842EC08BEF1A
:1030F000810F833098F52401350143E0440E511CC3
:10310000611C711C6D817E818F819885C2D98B83F2
:103110008115D9F0C301B201BCD98C83811571F03E
:103120008B819C8181305FEF950710F0982F882765
:10313000163071F0173079F00E947F262401350196
:1031400054E0450E511C611C711C5301420179CFA2
:103150000E942C26F3CF0E944D26F0CF143009F0A8
:10316000C1CF6D817E818F81988593D9182F2401DD
:10317000350184E0480E511C611C711CC501B4016D
:103180006D5F7F4F8F4F9F4F84D9111509F42DCE5E
:10319000811509F42ACE8150990B4FEF489F900179
:1031A000499F300D1124A12FA150BB0B2A0F3B1FAB
:1031B0002150310950F2EFE9FFE03197F1F700C0FB
:1031C0000000F6CFC6011DDCC0CF223009F07CCD57
:1031D00020918E0330918F03232B09F475CDFC01D0
:1031E000EE5DFB4F20812E7F2083835E9B4F0E94EC
:1031F000F4106ACD03375CE71507B9F480919403A6
:10320000811519F00E94CB0DF0CD1092A5040E94FB
:1032100077040E94B10888579C4E90939603809340
:10322000950381E080939403E0CD023A82E518078C
:10323000C1F158F4C80190528115904220F1013E2D
:10324000110579F1053E110503C0023BB2E51B07EC
:1032500009F03ACD25EE30E02770332781E090E089
:1032600001C0880F2A95EAF72091970330919403C3
:103270003115F9F0D70115963C913115A9F0282B9D
:1032800020939703B2CDF7018681803108F01CCDE1
:10329000812F99278F7199278230910511F04297DC
:1032A000D7CF21EE30E0D8CF80958223809397034B
:1032B0009CCD322F3823311509F406CD982F9095E7
:1032C0009223909397030E946F04F70185818115E3
:1032D00009F48BCDF9CC003EB2E51B0708F047C0DE
:1032E000003CE2E51E0728F5003AF2E51F07E8F486
:1032F000003622E51207E8F4C801925580349105A2
:10330000C0F01092A704C8018E32910508F063C086
:103310008832910508F050C08E31910508F04EC0FA
:1033200004974A9708F40ECD37C0043B32E51307E3
:1033300041F7F7013580311409F457C00E35FCE729
:103340001F0709F44EC00F352CE7120751F00D3559
:103350003CE7130709F049C080911001811509F479
:1033600040C01092100180E00E9419113ECD093733
:103370004CE7140728F407375CE71507D0F6C1CFF0
:103380000B378CE71807D4CF812F8F71843189F2E6
:10339000863111F41092A7040E94CB0D80919703FF
:1033A0000E946904C6CFD70116968C91803108F02F
:1033B000C1CCBFCFC801C0CC8A9771F78091970369
:1033C000811531F08091A70492E089278093A704AA
:1033D0000E949D0CAECF8C34910581F38D329240CA
:1033E000ECCF81E08093100100CD8091100181111C
:1033F00069C0C80197558115914008F0FFC0580178
:10340000F8EFAF22BB24A114B10409F0EECCF8010F
:10341000FF2754E0EE0FFF1F5A95E1F79F01235E4F
:103420003B4F6901D70115968C91EE5DFB4F908162
:1034300080FB90F99083811509F4D9C10E94B108ED
:103440009093A00480939F04F60182818F5F828312
:103450008091A7049091A504892B83838091A40473
:1034600084834681578166857785C6010E94EA0775
:10347000D60115968C9181FF5801B0929E04A092BE
:103480009D04D70115969C91911509F419C61092C7
:10349000A104980130572332310508F01FC684E09B
:1034A00090E00E94813190935F0580935E05F80162
:1034B000E150F047E232F10508F0E1C1E751FE4C7E
:1034C0000C94E430380150EE651A71085090A6044F
:1034D0008091A504582A8091A404582A88E068168F
:1034E000710408F05EC098012770332781E090E0F6
:1034F00001C0880F2A95EAF7311409F44FC0582A01
:10350000D7018D919C910E94F10321E030E0F901F7
:1035100002C0EE0FFF1F8A95E2F7FA87E987209134
:103520001304309114043E832D8340911B04509169
:103530001C045C874B876AE9C62E63E0D62EA12C5B
:10354000B12C511005C0D60112968C9181111BC06F
:10355000F601838190E029853A8582239323892B84
:1035600091F08085982F9770911101C087E038E025
:103570006316710408F066C0311409F45FC08695C3
:103580008170811164C09FEFA91AB90AAFE0CA0E19
:10359000D11CB8E0AB16B104A1F61CC0809558222E
:1035A000AFCF311038C080911B0490911C040817D4
:1035B000190781F410921C0410921B041092170436
:1035C000109218041092190410921A041092160402
:1035D000109215048091130490911404009709F43B
:1035E00008CFE8E06E16710408F0EBC0652D0E946C
:1035F0002907811103C081E00E941911F70185811B
:10360000F801E851FC47E730F10508F03ACFE55FF3
:10361000FD4C0C94E43010931C0400931B040E9496
:10362000080A609317047093180480931904909308
:103630001A04109216041092150462CF82FB882798
:1036400080F99FCF311409F49ECF80FF9CCFD60123
:103650008D909C900815190519F4311409F493CF35
:10366000ED81FE81EC15FD0509F48DCFD6011D9687
:10367000ED91FC91309721F08081811509F483CF81
:10368000652DC6010E942907811509F47CCF81E0D0
:103690000815190509F080E0482E43208114910493
:1036A00041F0411006C0EB85FC858E169F0609F09F
:1036B0006ACF80E00E941911D0921404C0921304C2
:1036C00081E0809312048FE08A9DF0018B9DF00DC4
:1036D0001124E656FC4F85818093990341100EC05A
:1036E0008114910459F0808191819C012450310909
:1036F000213A310508F049C00E9482088FE08A9D76
:10370000F0018B9DF00D1124E656FC4FC680D7804A
:10371000C6019A9581159F4110F420EED22299247A
:103720009394C60101978F339E4708F0912C8FE048
:103730008A9DD0018B9DB00D1124A656BC4F1996C1
:10374000ED91FC911A97309731F01B966D917C9119
:1037500081E0099598229114A9F08FE08A9DF001EB
:103760008B9DF00D1124E656FC4F868197810E94B7
:10377000540380939803C60148E06416710440F432
:103780000E94140A0E949D0C0AC00E947A0DB6CFB6
:103790000497813A910548F48C2D0E944E084114FB
:1037A00009F427CE0E949D0C20CB0E949D0C8FE334
:1037B0009CE90197F1F700C000008C2D0E94000DDC
:1037C000EECFDC012D913C910217130741F431102B
:1037D00009C01092120480E00E9419110ACE31141F
:1037E00009F407CEFC01808585FD03CEF4CFF901F5
:1037F0004485558566857785C9010E94EA07D6010B
:1038000015968C9181FF3DCEC6010E94D810809103
:103810009D0490919E040817190709F032CE10926A
:103820009E0410929D042DCE06E221EE41EE6AE147
:103830007CE728D8DACA07E225EE45EE6BE17CE7A3
:10384000F8CF06E221EE40EE68E17CE7F2CF07E236
:1038500025EE44EE69E17CE7ECCF06E221EE42EE94
:103860006CE17CE7E6CF07E225EE46EE6DE17CE712
:10387000E0CF08E221E045EE6EE17CE7DACF80910F
:103880005E05816080935E0560915E0570915F05C5
:1038900084E090E00E94AF310E94D40DA6CA8091CE
:1038A0005F05886080935F05EFCF80915E05826041
:1038B000E9CF80915E058460E5CF80915E058860E8
:1038C000E1CF80915F058160EDCF80915F058260DF
:1038D000E9CF80915E058061D5CF80915E058062E1
:1038E000D1CF80915E058064CDCF0E94D40D8091B0
:1038F0005E058068C7CF80915E058C60C3CF8091E4
:103900005F058360CFCF80915E058E7FBBCF8091B6
:103910005F05877FC7CF80915E058D7FB3CF809194
:103920005E058B7FAFCF80915E05877FABCF8091A7
:103930005F058E7FB7CF80915F058D7FB3CF80917C
:103940005E058F7E9FCF80915E058F7D9BCF80919E
:103950005E058F7B97CF0E94D40D80915E058F7797
:1039600091CF80915E05837F8DCF80915F058C7FA5
:1039700099CF80915E05992782FF939590FB82F9FC
:1039800090FB83F97FCF80915F05982F909590FBF6
:1039900080F990FB81F986CF90915E05892F8F7B0E
:1039A00096FF80646FCF0E94D40D90915E05892FA1
:1039B00097FB87F9805866CF61E08EE090E00E9427
:1039C000953162CF60E0F9CF90915E05892F8F7EAF
:1039D00094FF806157CF90915E05892F8E7F90FF75
:1039E000816050CF90915F05892F877F93FF88601A
:1039F00059CF89E285C389E26EC30737BCE71B074D
:103A0000F9F00837ECE71E0731F19801205E3245E6
:103A10002032310528F5911123C00F7181E090E02B
:103A20009C0102C0220F331F0A95E2F78901622F21
:103A300083E090E00E949531802F0E949D03D5C9BC
:103A400081E0911551F00E94A30343E062E081E020
:103A50000E942504CAC982E0F4CF0E94AD03F5CFCD
:103A60004091A30480915D05282F30E0209530958A
:103A700070E024233723232B19F048234093A30419
:103A80000B373CE7130741F4911509F4AEC90E94C6
:103A90008A030E944A07A9C9003442E5140708F0C6
:103AA00055C0003252E5150708F057C0011580E5F2
:103AB000180750F50115A0E41A0708F064C0911525
:103AC00009F479C00A35FCE71F0709F4CDC008F0F6
:103AD000B2C001303CE7130709F4C4C003304CE71F
:103AE000140709F4B9C001151C4709F064C00E940D
:103AF000D40DAFEFB4E3ECE0A150B040E040E1F70B
:103B000000C000000E94D40B9801305521153240AE
:103B1000B0F6980145E0369527954A95E1F7822F52
:103B20008F702091A30430E041E050E0082E02C0E5
:103B3000440F551F0A94E2F724233523232B09F45D
:103B4000BECF9111A6CF1092A5042CCE9801205C77
:103B500032452032310508F0B2CF802F8F7120918D
:103B6000A30430E041E050E0082E02C0440F551F8E
:103B70000A94E2F724233523232B09F4A0CF9115CF
:103B800009F433C986CFF7018681803108F097CFD9
:103B9000911111C0212F2F7081E090E002C0880F99
:103BA000991F2A95E2F72091A30430E08223932302
:103BB000892B09F01AC9F70187819085009709F4CC
:103BC00057C00E9475058C01F701B580A680A294AC
:103BD0002FE0A2228091A8048770811501F1CB2CDF
:103BE000B114F1F0812F807F803461F080E2800F8A
:103BF0008830A8F0812F807E803221F4023078F066
:103C0000A11469F080915F0582FF09C082E00E94E3
:103C10004E048091A8048770CC24C3948111C12CD8
:103C2000E12FE295EF70103C08F094C0F0E0EE5EFA
:103C3000FD4C0C94E4300B358CE71807B9F08091FB
:103C40005F05002482FF0394802D0C351C4709F08A
:103C5000B2CF0E945F0CAFCF6FEF7FEF80E090E0BC
:103C60000E94AF310E94000E81E0F3CF80E0F1CFDF
:103C70008581C080D180811569F0C6010E94BE1186
:103C8000182F682FC6010E94BB03B601812F0E9426
:103C9000A31197CFC6010E94F103182FF6CFF12F81
:103CA000FF70DF2E103118F0D29490EFD922B114AA
:103CB000A9F0D11459F080E2800F883010F0011182
:103CC00007C08D2D0E9469040E949D0C802F40C06A
:103CD0008091A7048D298093A704F6CF802F0E949E
:103CE0007A0DD114B9F180E2800F883010F0011103
:103CF00004C08D2D0E946F0406C0D0948091A7044B
:103D00008D218093A7040E949D0C24C0212F2F7029
:103D1000D22E107F103219F0D29480EFD8220115E4
:103D200049F0013009F483C0B11409F48FC0A11423
:103D3000A9F1CCCF80915F0582FD2CC0B11421F197
:103D4000D11429F08D2D0E9469040E949D0C80E001
:103D50000E94000DC11409F4D9C08091A80480FD0F
:103D6000D5C0D70115961C928695869586950E949A
:103D7000A303C7010E94AF158091A804869586957C
:103D800086950E94AD03C2C080E00E947A0DD114D6
:103D900009F3AFCFB11469F1A11004C08D2D0E94B9
:103DA000F10CD8CF31E0A31210C01091A4048D2DD6
:103DB0008123D81679F20E94B1089093AC048093C5
:103DC000AB041D291093A404C5CF45E0A412C2CFB3
:103DD0008D2D0E94F10C8D2D0E940F098091A6045B
:103DE0009D2D9823D91609F4B5CF8D298093A6046B
:103DF000B1CFA11012C08D2D0E94BB0D8D2D0E9440
:103E00000F098091A6049D2D9823911509F4A2CF46
:103E1000D094D822D092A6049DCF51E0A5129ACF7B
:103E20008091A5048D21811509F494CFE4CFB114BC
:103E300029F086E0A81608F08DCFB0CF95E0A9163E
:103E400008F088CF8D2D0E94BB0D84CFA114D1F333
:103E5000093349F4AFEFB7EEE3E0A150B040E040E2
:103E6000E1F700C00000802F0E947A0D73CF812FF0
:103E7000869586958370811561F0813009F06ACF4F
:103E8000C8019370B11002C080E090E00E94260843
:103E900061CFC8019370B11002C080E090E00E9431
:103EA000FE0758CF6B2D802F0E944D0953CF812FD5
:103EB0008370811139C0B11027C0402F42954695BB
:103EC0004770440F440F802F8F70042E01C0880F5D
:103ED0000A94EAF7202F207104FF07C02FE030E09A
:103EE00001C0220F4A95EAF7209516951695137092
:103EF0001230A9F0133089F030915C05113061F077
:103F0000822B83230E949D030E94EF0760E0C7017C
:103F10000E94E8110C940617832B822BF3CF822B7F
:103F200090915C058927EECFB11451F110FFECCFD1
:103F3000402F429546954770440F440F802F8F7055
:103F4000042E01C0880F0A94EAF7202F207104FF85
:103F500007C02FE030E001C0220F4A95EAF7209514
:103F6000169516951370123089F0133069F0309160
:103F70005D05113041F0822B83230E94A003C4CF42
:103F80008230B0F6C1CF832B822BF7CF822B90915A
:103F90005D058927F2CF1F70B11439F0812F0E947F
:103FA000A303802F0E94F10CAFCF802F0E94BB0D86
:103FB000812F0E94AD03A8CF023F71F170F4003F42
:103FC000C9F0013F91F0B11409F465C0A11409F4DE
:103FD0005FC0802F0E94000D97CF033F21F1043F67
:103FE00091F780915F0582FD2AC0812F8F71B114F6
:103FF00001F316C0B11469F0F5E0AF1608F084CFF4
:104000001F7181E090E0012E01C0880F0A94EAF749
:10401000BECF26E0A216F2CF812F8F71B110C9CF8B
:104020000E94A30371CF80E0B11409F4A6CF1F71E1
:1040300081E0012E01C0880F0A94EAF79ECFB114E7
:10404000C1F08091A8048770843049F41092A804CC
:104050001092AA041092A904812F8F71AACF35E083
:1040600063E0A31608F050CF812F8F710E94FB08E8
:104070004BCF45E0A41640F01092A8041092AA0479
:104080001092A90464E0F0CF81E00E944E043CCF7E
:10409000812F8F71C5CFA114F9F2093349F45FEF75
:1040A00087EE93E0515080409040E1F700C000005F
:1040B000802F0E947A0D28CF0337BCE71B0708C961
:1040C0000631FCE71F0709F098CC8091A204811506
:1040D00009F491CC85E30E94820864CB06312CE779
:1040E000120709F08ACC8091A5048A7A91E08111A7
:1040F00001C090E09093A204811509F47ACC85E385
:104100000E944E084FCBA0E0B0E0E9E8F0E20C944A
:104110000C3180910303803108F049C08091020383
:10412000811509F444C0C091B40289E0D82E809171
:10413000B3028C17E1F1EC2EF12CDC9EE00111248E
:10414000FE01EB54FD4F84818115B1F19181809185
:10415000FE02981331C090818091FD0298132CC00B
:104160008581811129C0028113818091FF02909184
:104170000003081B190B60E08DEF92E00E94E8112C
:104180000E94271408171907B8F4809103038F7051
:10419000806180930303C554DD4F88818F708061F7
:1041A00088838DEF92E00E94AF150E944404CDB742
:1041B000DEB7E7E00C942831E7012196C770B7CF4E
:1041C000AFE0B0E0E6EEF0E20C9404318C0186E062
:1041D000F801DE011A9601900D928A95E1F7F80137
:1041E000F580E4808DEF882E82E0982E8091010387
:1041F000811117C0E11491F0F11409F480C1C801D4
:104200000E941712811509F47AC189E0F801ADEF17
:10421000B2E001900D928A95E1F775DFFF24F394E7
:104220006AC0A280B380D09002038091FF02909177
:1042300000033501681A790AD11409F411C1C0804C
:10424000518060E08DEF92E00E94E8110E942714F7
:104250006816790608F0B6C0E11401F38091FE02F9
:10426000F8019181E0900303F0E1EF1608F064C0DB
:10427000981320C09091FD02F801808198131AC014
:104280002091040330910503878190852817390711
:1042900089F4F1104BC08E2D8F70806180930303E1
:1042A0008DEF92E00E94AF1580910303F8018683A1
:1042B000F12C21C0F1103AC040E0652D8C2D0E94F8
:1042C000B50B40E0652D8C2D0E94B50BF82E8111A9
:1042D000EFCF8A859B850E940A12292F22952F7085
:1042E000903470F49F702230A0F09115B1F0F80175
:1042F0009681903190F48F2D2F96EFE00C94203121
:104300002A5F2F70223068F0C8010E94AF15FD2C83
:10431000F2CF911511F0811571F3805E883058F35A
:10432000F3CF803F40F3815F8330F9CF8091030367
:10433000816080930303BCCF98131EC09091FD024F
:10434000F8018081981318C020910403309105036F
:10435000878190852817390779F4F1100DC0E6821E
:10436000C8010E94AF1589E0F801ADEFB2E00190FD
:104370000D928A95E1F752CFC8010E94171281155C
:1043800009F4BDC0F11409F4BAC08091030380326E
:1043900008F43BCF8091FD029091FE029A838983BD
:1043A000BC82AB82809101038D831E82EF8280915B
:1043B00004039091050399878887CE0101960E9496
:1043C000AF1523CFD0900303F0E1DF1650F48DEF4B
:1043D00092E00E94AF1589E0F40111928A95E9F705
:1043E00067CFE11409F41ACF9091FE02F8018181A0
:1043F00098131AC09091FD028081981315C02091E6
:10440000040330910503878190852817390761F4EB
:10441000F1100AC0D682C8010E94AF1589E0F401EC
:1044200011928A95E9F7FACEC8010E9417128115F8
:1044300009F465C0F11409F462C08091030380326D
:1044400008F4E3CE8091FD029091FE029A83898365
:10445000BC82AB82809101038D831E82DF82A7CF55
:1044600060E08DEF92E00E94E8110E942714681628
:10447000790608F0B0CFE11409F4D0CEF11409F4B4
:104480003EC09091FE02F801818198132EC0909158
:10449000FD028081981329C0209104033091050307
:1044A000878190852817390701F58091FF02909147
:1044B0000003A81AB90AF8ECAF16B10408F053CFFC
:1044C0008091030380FD4FCF803108F44CCFF80179
:1044D0008683982F907F903F09F442CF982F907F4A
:1044E000905F8F70892B86833BCFC8010E94171283
:1044F00081118BCE80910303816080930303C801F7
:104500000E94AF158BCEA2E1B0E0E9E8F2E20C9494
:104510000F310A871B872C873D874E875F87688B03
:10452000798B8A8BCE010A964BDE811128C02091AF
:10453000B3023091B40289E0FE013A96DE01119691
:1045400001900D928A95E1F78E858115C1F0822F39
:1045500090E001968770992738171906D9F099E0ED
:10456000929FD0011124AB54BD4FFE0131960190B2
:104570000D929A95E1F78093B3020E94440419E0EA
:104580008091B4029091B302891312C06296E4E064
:104590000C942B310E94D40D1092B3021092B402ED
:1045A00089E0EDEFF2E0DF011D928A95E9F7E7CFB0
:1045B000189FC00111248B549D4F02DE811531F3E9
:1045C0008091B40290E00196877099278093B4029D
:1045D000D7CFEF92FF920F931F93CF93DF938091EA
:1045E0005905E091F401CDE0811130C0CDB7DEB7BF
:1045F000E6E00C942931D1E0DE0FD093F401EE2EE9
:10460000F12CCE9FF0011124EF50FB4F84818115D6
:10461000E1F087819085892B21F48185928501962F
:1046200051F4008111812281338144815581668159
:104630007781808568DFCE9DF001CF9DF00D11243C
:10464000EF50FB4F14821092A704ED2F8091590573
:10465000E81788F2109259051092F401C7CFA4E030
:10466000B0E0E5E3F3E20C9402312091F0042983F9
:1046700097E0992E01E010E02DE0322E34E0532E29
:10468000882483948091EF049981891307C0A1DF66
:104690000E94EC062496E1E10C941E319981892F49
:1046A00090E09C838B83FC01EE0FFF1FEB51FB4FCF
:1046B00080819181989ED001999EB00D1124FD01B9
:1046C000E355FB4FFA83E983248121115BC060909D
:1046D0005905E1EFF4E060E070E0712C661508F038
:1046E0004FC0A384B484A981BA81CD90DC902FEF10
:1046F0003FEF412C442D50E07601E40CF11CE40C1A
:10470000F11CD701ED90FC90E114F10439F0AE14E6
:10471000BF0409F0A90143949A01ECCF2F3F32075F
:10472000D1F1D80102C0AA0FBB1F2A95E2F77A2A5D
:104730009801042C02C0220F331F0A94E2F7A9014A
:10474000415051097416150629F5369EF001379E21
:10475000F00D1124EF50FB4F989ED001999EB00DA3
:104760001124A355BB4F12962D913C91139730877E
:1047700027835482108211829287818715968C92AA
:104780000E94FD068B819C8101969A8389838370A8
:10479000898378CF14826F5F7F4F3D969FCF1092B1
:1047A0005B0510925A05109211018091EF048093DD
:1047B000F0040E94EC060DCFACE1B0E0E2EEF3E2D3
:1047C0000C9401314B8B5C8B6D8B7E8B8F8BB92E58
:1047D000988FA92E91111092A704188A198A1A8A03
:1047E00086E0FE017396DE011A9601900D928A957D
:1047F000E1F75F8880915F0582FF1FC00E94B108CA
:104800002091A9043091AA04821B930B883893410C
:1048100038F08091A80482FD03C082E00E944E041B
:104820000E94B1082091AB043091AC04821B930B21
:104830008838934110F00E9477045114D9F05E86B5
:10484000BF8661E0CE010A960E94E81161E0CE01C8
:104850000A960E94E81161E0CE010A960E94E811D2
:104860004C0180356CE7960791F4A11419F181E0B1
:10487000809311015E86BF860A851B852C853D8548
:10488000452D5B2D688979898A893DDECDC08135CA
:104890009C4721F4A11471F082DFECCF82E58816E9
:1048A0008CE7980639F4A11429F080911101811147
:1048B000F3CFDDCF4DEAE42E44E0F42E412C612C01
:1048C000712CD7016D917C91CC24CA94DD24DA94AB
:1048D00080E0282F30E0FB01E80FF11DE80FF11D0B
:1048E000408151814115510539F08416950609F032
:1048F00096018F5F6901EDCF10E0BFEFCB16DB06AD
:1049000009F44EC0F701448110911101411110E0EA
:10491000D70115963C90159716969C911697A11461
:1049200009F405C1111509F402C1311017C021E0C5
:1049300030E00C2C01C0220F0A94EAF7922B169655
:104940009C932091ED043091EE042233310530F434
:1049500022E330E03093EE042093ED04E1E0F0E058
:1049600002C0EE0FFF1F8A95E2F7CF010197D70132
:1049700016962C912817190699F4C0905A05D090D4
:104980005B05C114D10409F453C00E94B1088C190D
:104990009D09C39708F44CC081E0F701848311E0BE
:1049A000412ABFEF6B1A7B0AE7E0EE0EF11CF8E03C
:1049B0006F16710409F085CFA11409F417C14114D1
:1049C00009F414C10E94B10890935B0580935A05C5
:1049D00080915905883040F591E0980F90935905E2
:1049E00099E0FE013A96DE01119601900D929A959A
:1049F000E1F75D82BE822DE0829FC00111248F50BD
:104A00009B4F29E0FE013196DC0101900D922A9521
:104A1000E1F72FEF3FEFDC011A963C932E931997A5
:104A20001C969C928E921B976C96E2E10C941D3121
:104A30002091F0048091EF04922FE0E0F0E001E09B
:104A4000281709F448C0422F50E0FA01EE0FFF1F6B
:104A5000EB51FB4F2080318037E0329DF001339DD8
:104A6000F00D1124E355FB4F608171817C8F6B8FBA
:104A7000B0E030E0A0E0EB8DFC8DEA0FF11DEA0F15
:104A8000F11DC080D180C114D104E1F0F701019083
:104A9000F081E02DFA8FE98F30E007C0E1E0C61623
:104AA000D70609F0E0E0BE2B3F5FE98DFA8DE30FFA
:104AB000F11DE30FF11D608171816115710571F7C1
:104AC000AF5FD9CFB11581F13A17C8F4E1E0D70152
:104AD0001496EC93F7019093F004EE15FF0509F49A
:104AE0005FCF90E0FC01EE0FFF1FEB51FB4F718297
:104AF00060820196837099278093EF0451CF37E04D
:104B0000329DF001339DF00D1124E355FB4F0483DA
:104B1000EE15FF05F9F2291302C09F5F93709A0109
:104B20002F5F3F4F23708CCFE0E0F0E0F8CF292FCC
:104B300030E0311024C061E070E002C0660F771FE2
:104B40008A95E2F7CB0101972817390791F010E019
:104B5000E1E0F0E002C0EE0FFF1FCA94E2F76F0140
:104B6000C094D70116968C9116978C2116968C932B
:104B700017CF411569F3C3010E94FD06E8CFA901D3
:104B80000C2C02C0559547950A94E2F7C90101978C
:104B900082239323892B39F540FF25C0D701129634
:104BA0008D919C91892BD1F087E0FE013196DF0138
:104BB0001D928A95E9F70E94B1089C018B839C8322
:104BC00084E08D83F70192818381792F988789878B
:104BD00009811A8144E05E816F8195DCD7011596C9
:104BE0001C92132DB5CF142F1170B2CF9091F004F9
:104BF0008091EF04981731F032DDB1E04B1609F4E3
:104C000013CF38CEE6DC10925B0510925A050E9455
:104C1000EC06F3CFA6E0B0E0E0E1F6E20C940F3151
:104C20000E94B1088C0180918702909188028017C0
:104C3000910771F019821A820E94B108BC01498162
:104C40005A8180E090E0B8DD1093880200938702DB
:104C50002696E4E00C942B31A6E0B0E0E2E3F6E225
:104C60000C9411319093840280938302811520E289
:104C7000920730F40E94650D2696E2E00C942D31E7
:104C800080EF89838A830E94B1088160BC014981D9
:104C90005A8181E091E090DDEFCFA6E0B0E0E3E55E
:104CA000F6E20C940F318C0190938402809383027E
:104CB000011580E21807B0F4802F0E947A0DC80118
:104CC000805E9109089728F061EC7DE001151105DF
:104CD00011F46BEB7DE0C8010E947E032696E4E0B0
:104CE0000C942B3180EF89838A830E94B108816004
:104CF000BC0149815A8181E090E05EDDEFCFCF9326
:104D0000DF93D82FC92FA8DF8D2F9C2FC6DFDF910F
:104D1000CF9108950F931F93CF93DF938C01862F2C
:104D20006AE873E00E941214892B91F4C0918A03FF
:104D3000D0918B03209761F0F8018281833039F4A0
:104D4000CE01DDDFCE01DBDFCE01D9DF01C0E0F730
:104D5000DF91CF911F910F9108950F931F93CF93E0
:104D6000DF938C01EB016AE873E08C2F0E94121430
:104D7000892B09F057C0FE01FF27D80112968C91AC
:104D80001297EA5BFD4F8130A9F415968C9182FD54
:104D90004EC080FF4CC082E0808380918C03909154
:104DA0008D030097B9F480918A0390918B0300974B
:104DB000C9F110C08230A1F515968C9182FD26C0F4
:104DC00080FD0AC083E0808380918E0390918F03E1
:104DD0000097F1F041DF26C084E08083809190034A
:104DE000909191030097B1F780918A0390918B0382
:104DF000009701F184DF80918C0390918D030097DF
:104E000049F780918A0390918B03E4CF85E08083FA
:104E100080918A0390918B03009721F070DFF1CF8E
:104E200086E08083DF91CF911F910F91089581E0FB
:104E30008083B9CF80918C0390918D03B8CF0F936D
:104E40001F93CF93DF938C01EB016AE873E08C2F03
:104E50000E941214892B71F4DD27CA5BDD4F888113
:104E6000F801128218828330E9F048F4813059F059
:104E7000823081F0DF91CF911F910F91089584309E
:104E8000B1F08530B9F780918A0390918B03009738
:104E900089F306C080918C0390918D03009799F35C
:104EA000FCDEE8CF80918E0390918F03F7CF809145
:104EB000900390919103009799F720918A03309184
:104EC0008B0380918C0390918D0321153105F9F2AC
:104ED000009731F7C901E4CFAAE0B0E0E2E7F7E2DA
:104EE0000C940531FE0131968AE0DF011D928A950E
:104EF000E9F79AE2A92E91E0B92E8F013F01EE2445
:104F0000E394F12C3DE3C32E31E0D32EF5018191E2
:104F10005F018F3F09F444C0F894E82FE295EF70E9
:104F2000F0E021A18F70A70102C0440F551F8A95A0
:104F3000E2F7CA01922F982B91A392A18095892321
:104F400082A3789400C0EFE2F1E021E030E0812C10
:104F5000912C41914F3F79F0A42FA295AF70A05EA4
:104F6000B0E08C9190E04F7002C0959587954A957E
:104F7000E2F780FF3BC080E090E0882A992A220F68
:104F8000331FCE16DF0629F7F50182918F3F11F00E
:104F90000E94730650EA5A95F1F7D8018D929C92BF
:104FA0000E5F1F4FBFE2AB16B1E0BB0609F0AECFFC
:104FB0004AE050E0B3018EE492E00E945531892B23
:104FC000B9F08AE0F301AEE4B2E001900D928A9567
:104FD000E1F781E08093D6010E94B1089093D5015A
:104FE0008093D4012A96EEE00C942131C901C5CFFB
:104FF0008091D6018115B1F30091D4011091D501B2
:105000000E94B108801B910B059760F34AE050E0C5
:105010006EE472E086E792E00E945531892B49F0F8
:105020008AE0EEE4F2E0A6E7B2E001900D928A9504
:10503000E1F71092D601D6CFCDB7DEB7AC970FB659
:10504000F894DEBF0FBECDBF85B7806885BF85B73A
:10505000806885BF84B7877F84BF0FB6F894A89512
:1050600080916000886180936000109260000FBEA4
:1050700080E890E00FB6F89480936100909361000F
:105080000FBE81E080930F0181E796E09093AB0122
:105090008093AA010E9499060E940F130E94531345
:1050A0000E94D2130E94FE0A0E945B0B8091E200D4
:1050B00084608093E200789480918202811599F057
:1050C0008091E9001091EC008F70179511271795CA
:1050D000182B1092E9008091E80083FD0E94150EC4
:1050E0001F701093E90082E084BD93E095BD9AEFB4
:1050F00097BD80936E000E945912811102C00E94D8
:10510000DC140AE211E0D8018D918D018F3F11F07E
:105110000E947306B1E00F321B07A9F70FE211E0FE
:10512000F80181918F018F3F11F00E947306F1E029
:105130000D331F07A9F78AE0E6E7F2E0DF01282F29
:105140001D922A95E9F7EEE4F2E0DF011D928A95BF
:10515000E9F780E090E00E948131833E9E4F21F488
:105160000E945912811129C063EE7EEF80E090E029
:105170000E94AF3160E082E090E00E94953181E0D2
:1051800080935C0561E083E090E00E94953160E0EF
:1051900074E184E090E00E94AF310E94DC1440E0B2
:1051A00050E0BA018FE090E00E94A73140E050E06B
:1051B000BA0183E190E00E94A73182E090E00E9472
:1051C000793180935A0284E090E00E94813190937B
:1051D0005F0580935E0580DEEFEFF6E721E0E150AA
:1051E000F0402040E1F700C0000076DE80917602BA
:1051F00080FF08C06FEF7FEF80E090E00E94AF314A
:105200000E94D40B83E090E00E9479310E949D03BC
:1052100080E091E09093AA028093A902809182029B
:10522000853049F480918202853009F45AC00E9489
:10523000D40D0E94EF0750DEEBE5AE2EE2E0BE2E6D
:1052400006E712E0D801F501219131918D919D91F0
:1052500042E0E536F40709F479C028173907A1F3CD
:1052600076E7872E72E0972E512CD401ED90FD90B9
:105270004D01F501619071905F016E147F0451F151
:105280006E247F24412CCC24C394D12CC3018C21C7
:105290009D21892BB1F049825A820E94B1089C83DA
:1052A0008B83F1E0FD8391E097012C213D21232B9D
:1052B00009F490E09E8349815A816B817C818D81C4
:1052C0007BDA4394CC0CDD1C2EE04212DFCFF501DB
:1052D000F292E292539435E05312C7CF0E94080A2B
:1052E0003AC080918202843021F11092580288E104
:1052F00090E0A0E40FB6F894A895809360000FBEEC
:10530000A093600083B7817F846083BF83B781608F
:1053100083BF7894889583B78E7F83BF0FB6F89448
:10532000A895809160008861809360001092600071
:105330000FBED2DDE6E7F2E081919191892B09F071
:1053400095C5B2E0E038FB07B9F76CCF28173907ED
:1053500009F086CF5FDCE0901504F0901604E114AC
:10536000F10491F18090690290906A02A0906B0222
:10537000B0906C020E94080A681979098A099B0991
:105380008090650290906602A0906702B0906802DB
:10539000681579058A059B05B8F0C7010E94650D5F
:1053A00010921604109215041092690210926A026B
:1053B00010926B0210926C021092650210926602BB
:1053C0001092670210926802C0909D04D0909E04D3
:1053D000C114D10439F1A0909F04B090A0040E94A0
:1053E000B1087C01EA18FB08C6010E9427148E153B
:1053F0009F05C0F420919D0430919E04C901992716
:10540000287F3327232B09F055C144E0880F991FCB
:105410004A95E1F7835E9B4FDC0115962C9122FFA4
:105420000E94F41080911101811511F1E0905A054C
:10543000F0905B05E114F104D9F00E94B1088E19D7
:105440009F092091ED043091EE042817390780F46C
:105450009091F0048091EF04981709F42EC1FFD8C1
:105460001092EE041092ED0410925B0510925A0512
:1054700080919403811569F00E94B10820919503F1
:1054800030919603821B930B8F3F9F4710F40E942D
:10549000CB0D86E0E4E2F3E0DE01119601900D927F
:1054A0008A95E1F790902503B0902603D0902703CA
:1054B000A0902803C090290310922603109227037E
:1054C00010922803109229038D2D8B29811509F440
:1054D00041C0E0906F02F09070020E94B1089C0100
:1054E0002E193F0990912203911509F4BAC4253170
:1054F000310580F19F3F19F09F5F90932203B11413
:1055000059F00E947F0791E01B140CF09FEF899FD8
:10551000802D112480932603D11459F00E947F0717
:1055200091E01D140CF09FEF899F802D1124809332
:10553000270380912603811569F0F0902703F11469
:1055400049F00E947107809326038F2D0E947107F6
:10555000809327038A2D8C29811509F441C0E0909E
:105560006D02F0906E020E94B1089C012E193F0955
:1055700090912103911509F46FC42135310580F113
:105580009F3F19F09F5F90932103A11459F00E944F
:105590009F0791E01A140CF09FEF899F802D112432
:1055A00080932803C11459F00E949F0791E01C14B6
:1055B0000CF09FEF899F802D112480932903809107
:1055C0002803811569F0F0902903F11449F00E9435
:1055D0007107809328038F2D0E9471078093290300
:1055E00080912503891119C080912603811511F03E
:1055F0008B1113C020912703211511F02D110DC01F
:1056000090912903911511F09C1107C03091280346
:10561000311103C0822B892B81110E94240986E05D
:10562000FE013196A4E2B3E001900D928A95E1F774
:105630000E94EF0790917102891721F08093710207
:105640000E94080A80918202843009F0E7CD83E04D
:105650008093E9008091E80082FFE0CD8091E8002E
:1056600090E085FF05C00E94CD0A811579F191E097
:105670008091E8008B778093E800911509F4CECDF6
:10568000E0908502F0908602E981E114F104E1F1F5
:10569000EE3F09F05CC08A81833020F08550833072
:1056A00008F055C0EA81EE3008F051C0F0E0E25E4B
:1056B000FD4C8AC580E090E0AFCE0E94E9221092B6
:1056C0005B0510925A050E94EC06D2CE30E2E32E22
:1056D000F12CFE0131966F018091E80085FD0AC032
:1056E0008091E8008B778093E8000E94CD0A8115B5
:1056F00099F3BDCF8091F100D6018D936D01B1E09A
:10570000EB1AF10849F7B3CFE43148F4E11551F051
:10571000E150E33138F4F0E0E45DFD4C55C5EE3F77
:1057200009F4C0CFEFEFE98312C01A8289E08B83BE
:105730000EC08A81823081F08330B1F0813091F7E0
:105740000E94080A57D56B837C838D839E83CE018C
:1057500001960E941D0B62CD88E290E0CAD51B82A3
:105760001C821D828E83F3CF8091800290918102F2
:10577000892B69F3FE013196D8018C9111969C9189
:105780000E5F1F4F928383833296B2E000381B076F
:1057900099F7DDCF8A81823049F46B817C818D81DC
:1057A0009E8128D588E290E0C0D5D1CF8FEF898344
:1057B000CECF4C816B818A810E94741198278927F2
:1057C00098279E838D83C3CF2D813E813227232747
:1057D00032274C816B818A810E94760CB8CF0E945F
:1057E0007212B5CF80E18A83B2CF1A8287E89FCF49
:1057F0008C818D3108F0ABCF8A809B8098248924DE
:105800009824A12CB12C9E012F5F3F4F7901890173
:10581000080F111D0E151F0509F499CF80E037E818
:1058200083169104A104B10420F4C40187589C4F4D
:1058300060D5D70114968C93BFEFEB1AFB0AEFEFFC
:105840008E1A9E0AAE0ABE0AE5CF80918002909120
:105850008102892B09F47BCF8C818D3108F077CFC1
:10586000882E912CA12CB12CCA80DB80DC24CD2485
:10587000DC24E12CF12C8E010F5F1F4F412C512CA9
:105880003201481459046A047B0408F060CFF7E839
:10589000CF16D104E104F10438F4D80114966C91C8
:1058A000C60187589C4F41D5BFEF4B1A5B0A6B0A64
:1058B0007B0AEFEFCE1ADE0AEE0AFE0A0F5F1F4FD9
:1058C000E0CF0E94A21443CF84E08DCF8C818D3134
:1058D00008F03DCF882E912CA12CB12CCA80DB8002
:1058E000DC24CD24DC24E12CF12C412C512C320180
:1058F0008E010B5F1F4F481459046A047B0408F0A3
:1059000026CF80E0F0E3CF16F2E0DF06E104F104F9
:1059100018F4C6018996EDD4D8018D938D01BFEF9F
:105920004B1A5B0A6B0A7B0AEFEFCE1ADE0AEE0A0D
:10593000FE0AE1CF2C81022F10E02D3108F007CFB5
:105940008A819B819827892798272C01612C712CAB
:105950008033F2E09F0708F0FACE822E912CA12C22
:10596000B12C40E352E060E070E04419550966094B
:105970007709421751056105710508F4E8CE2091B9
:10598000800230918102232B09F03EC01C0129E2E4
:10599000220E311C80FBEE24FF24E0F880FF0BC0B8
:1059A0008896A7D49D8189279827892781159C47A8
:1059B00011F48FEF8D83D501C401840D951DA61DB3
:1059C000B71D80FF19C0680141E0C41AD108CE019B
:1059D00005968C0D9D1D9CA78BA7C101800F911F63
:1059E00088D4ABA5BCA59C9181159C4721F48FEF71
:1059F000EBA5FCA580838601FE013196EE0DFF1D0F
:105A00002FEFE016F10638F08E010F5F1F4FC12C0B
:105A1000D12C760125C09481858181159C4711F494
:105A20002483258342E0E40EF11C3296EACF80E322
:105A3000481682E058066104710430F4D8011496C7
:105A40006C91C201899671D4BFEFCB1ADB0AEB0AC5
:105A5000FB0AEFEF4E1A5E0A6E0A7E0A0F5F1F4FB7
:105A6000C814D904EA04FB0410F371CE80918002BB
:105A700090918102892B09F46ACECE0101960E9491
:105A80001D0BFFEF21EE34E0F15020403040E1F7F4
:105A900000C00000B5CB88E0E2E1F1E0DE019196C4
:105AA00001900D928A95E1F7FE0132968FE1DF01B8
:105AB0001D928A95E9F786E0898388E07F96DE016A
:105AC000159601900D928A95E1F741CE88EC898375
:105AD00081E08A831B821C823ACE8B819C81092EB5
:105AE000000CAA0BBB0B25E0880F991FAA1FBB1F38
:105AF0002A95D1F7AC01BD01405E5F4F6F4F7F4FDC
:105B0000481759076A077B0708F421CE883CE1E073
:105B10009E07A105B10508F01ACE493CF1E05F07E8
:105B20006105710520F048EC51E060E070E0481B31
:105B3000590BBC01635C7B4FCE010196ADD307CE00
:105B40004AE150E06FEF70E0CE010796BBD3809141
:105B500080028983EA821B821C8284E08D838DE02F
:105B600001CE81E090E0909386028093850282E3EB
:105B700090E090937502809374020E94B108909314
:105B8000730280937202E3CDE114F10481F1D090AD
:105B90007602C0907F0200917202109173020E94FF
:105BA000B108801B910B8536910540F1C5FE26C0DA
:105BB000D0FE24C00E94B1089093730280937202B9
:105BC0008091740290917502019790937502809371
:105BD0007402892B61F4109286021092850281E092
:105BE00090E09093810280938002E12CF12C8091CF
:105BF00080028983EA828091740299CD82E390E0E9
:105C00009093750280937402F2CF109281021092E9
:105C100080029DCD40E250E06FEF70E0CE01019632
:105C200051D395CDEB81E93008F091CDF0E0E15C06
:105C3000FD4CCAC2FE0135968BE1DF011D928A95AB
:105C4000E9F788E089838A838B838C8383E088A348
:105C50007ECD8C819AE0F92E8E010F5D1F4FF801E9
:105C60002F2D11922A95E9F7B8010E941214898309
:105C7000F801DE01129601900D92FA94E1F767CDDA
:105C80001C818AE0FE013596DE01919601900D920D
:105C90008A95E1F789A19AA10E948C069AA389A30B
:105CA0008BA19CA10E948C069CA38BA38DA19EA17D
:105CB0000E948C069EA38DA38FA198A50E948C069E
:105CC00098A78FA38FEF183060F43AE0139FB001CC
:105CD0001124675A7D4F4AE050E0CE01819643D3AC
:105CE00080E089830E94990632CD2C816AE0CE0142
:105CF0008196DC01E62F1D92EA95E9F7283008F03D
:105D000044C0629FB001112467557D4F4AE050E0C6
:105D1000E0D280E089838AE0FE01B196DE0112962E
:105D2000D0CE1C818AE0FE013596DE01919601906D
:105D30000D928A95E1F789A59AA50E948C069AA7EB
:105D400089A78FEF183060F4FAE01F9FB00111248B
:105D500067557D4F4AE050E0CE01819604D380E044
:105D600089830E940F13F3CC2C816AE0CE018196C7
:105D7000DC01E62F1D92EA95E9F7283030F4629FA6
:105D8000B001112467507D4FC1CF8FEFC3CF1C816D
:105D90008AE0FE013596DE01919601900D928A957A
:105DA000E1F78BA19CA10E948C069CA38BA38FEF93
:105DB000183060F4FAE01F9FB001112467507D4F46
:105DC0004AE050E0CE018196CED280E089830E94E5
:105DD0005313BDCC2C8166E0CE018196DC01E62F09
:105DE0001D92EA95E9F7283060F4629FB001112412
:105DF000675B7C4F46E050E06CD280E0898386E0B0
:105E00008BCF8FEFFBCF1C8186E0FE013596DE0144
:105E1000919601900D928A95E1F789A19AA10E942D
:105E20008C069AA389A38BA19CA10E948C069CA39B
:105E30008BA38FEF183060F4F6E01F9FB0011124A0
:105E4000675B7C4F46E050E0CE0181968CD280E0CB
:105E500089830E94D2137BCC2B30310508F092CB82
:105E6000BFCB2B30310508F047CB74CB8091590262
:105E7000811509F4D7C9E0E1E9BDF2E1F9BD09B442
:105E800000FEFDCF8091D8008F7D8093D800809157
:105E9000E00082608093E0008091E00081FDFCCF13
:105EA0000E94D40DBFC91F921FB61F9211248F9359
:105EB0009F93AF93BF9380915802811113C080913B
:105EC000EC019091ED01A091EE01B091EF014196AE
:105ED000A11DB11D8093EC019093ED01A093EE0103
:105EE000B093EF01BF91AF919F918F911F901FBE13
:105EF0001F90189578941F921FB61F9211248F93AC
:105F00009F93AF93BF938091EC019091ED01A0918D
:105F1000EE01B091EF010196A11DB11D8093EC013E
:105F20009093ED01A093EE01B093EF01BF91AF917B
:105F30009F918F911F901FBE1F9018951F920F92D7
:105F40000FB60F9211242F933F934F935F936F934C
:105F50007F938F939F93AF93BF93EF93FF93809122
:105F6000E10082FF09C08091E20082FF05C08091BC
:105F7000E1008B7F8093E1008091DA0080FF24C0F4
:105F80008091D80080FF20C08091DA008E7F8093BE
:105F9000DA008091D90080FFA9C080E189BD82E14B
:105FA00089BD09B400FEFDCF81E08093820280911B
:105FB000DB01811109C00E94FE0A0E945B0B8091E7
:105FC000E20084608093E2008091E10080FF1AC0CB
:105FD0008091E20080FF16C08091E2008E7F809366
:105FE000E2008091E20080618093E2008091D8001D
:105FF00080628093D80019BC85E08093820283E0A0
:1060000080930F018091E10084FF2FC08091E20016
:1060100084FF2BC080E189BD82E189BD09B400FE07
:10602000FDCF8091D8008F7D8093D8008091E100D2
:106030008F7E8093E1008091E2008F7E8093E2006A
:106040008091E20081608093E2008091DA01811505
:1060500009F452C084E080938202809182028430ED
:1060600009F052C082E080930F018091E10083FF2C
:106070002CC08091E20083FF28C08091E100877FDF
:106080008093E10082E0809382021092DA01809195
:10609000E1008E7F8093E1008091E2008E7F80930B
:1060A000E2008091E20080618093E20042E060E0E3
:1060B00080E00E942B0B8091F00088608093F000BC
:1060C00081E080930F0180930E01FF91EF91BF91CA
:1060D000AF919F918F917F916F915F914F913F9180
:1060E0002F910F900FBE0F901F90189519BC109212
:1060F00082021092DB0168CF8091E30087FF02C02B
:1061000083E0A9CF81E0A7CF81E0ADCF1F920F92AE
:106110000FB60F921124EF92FF920F931F932F93BC
:106120003F934F935F936F937F938F939F93AF931F
:10613000BF93CF93EF93FF9309EE10E0F8018081B6
:10614000C091EC008F70C795CC27C795C82B1082E3
:1061500080EFE82EF12CF7018081877F808378948F
:106160000E94150EF8011082F701808188608083FB
:10617000CF70F801C083FF91EF91CF91BF91AF91A4
:106180009F918F917F916F915F914F913F912F914F
:106190001F910F91FF90EF900F900FBE0F901F90E7
:1061A000189597FB072E16F4009406D077FD08D0BB
:1061B0005FD007FC05D03EF4909581959F4F0895E0
:1061C000709561957F4F0895EE0FFF1F0590F49134
:1061D000E02D0994082E817006940694811D069482
:1061E000811D0694811D0694811D0694811D0694CF
:1061F000801D08956927962769277827872778279C
:1062000008952F923F924F925F926F927F928F925A
:106210009F92AF92BF92CF92DF92EF92FF920F9335
:106220001F93CF93DF93CDB7DEB7CA1BDB0B0FB63F
:10623000F894DEBF0FBECDBF09942A8839884888FC
:106240005F846E847D848C849B84AA84B984C88492
:10625000DF80EE80FD800C811B81AA81B981CE0F89
:10626000D11D0FB6F894DEBF0FBECDBFED0108956E
:10627000AA1BBB1B51E107C0AA1FBB1FA617B7076C
:1062800010F0A61BB70B881F991F5A95A9F7809588
:106290009095BC01CD010895FB01DC0102C0059081
:1062A0000D9241505040D8F70895FB01DC0104C025
:1062B0008D910190801921F441505040C8F7881BFE
:1062C000990B0895DC0101C06D9341505040E0F7F7
:1062D0000895DC01CB01FC01F999FECF06C0F2BDA7
:1062E000E1BDF89A319600B40D9241505040B8F794
:1062F0000895F999FECF92BD81BDF89A992780B58E
:106300000895A8E1B0E042E050E0E5CFDC01A40F41
:10631000B51F4150504040F0CB01840F951F2E9186
:1063200005D041505040D8F70895262FF999FECF57
:1063300092BD81BDF89A019700B4021639F01FBAD8
:1063400020BD0FB6F894FA9AF99A0FBE08950396F5
:10635000272FECDFEADF252FE9DF242FE7CF019697
:10636000272FE4DFE2CFDC01CB0102C02D9105D065
:1063700041505040D8F70895262FF999FECF1FBA03
:1063800092BD81BD20BD0FB6F894FA9AF99A0FBE5E
:1063900001960895F894FFCF59095E0960096509CF
:1063A00075097509750975097509750975097509FD
:1063B00067096B096E097309830989098D09F20E52
:1063C000180F1E0F180F1E0F700F910F1E0F971032
:1063D000A410831CEB1C8B1C551C591C8F1C5D1CB2
:1063E000931C9F1C691CE41C6D1CA31C711CA71C26
:1063F000CC1C751CAB1CD31C7B1CB11CB91C611CB8
:10640000971C651C9B1C7F1CB51CC31CDC1CE21C60
:106410004F1C871CF21C211C271C141C1B1C2D1C30
:10642000331C391C4F1E4F1E861E861E371F521FDF
:10643000AA1EAA1E571FCB1FDC1FDC1F4B2D662D6B
:106440006D2DA72BA72BA02DB12DC42D052E0A2E07
:10645000A72BA72BA72B122E952B992BCA2BD92B09
:10646000E42BEF2B922B922B922B922B362DF22B8F
:10647000F52BF82B252C612C642C662C9A2C1A2ECB
:10648000292E402E752E912EB42EC72EEA2E032FC4
:10649000AE083A0C500C550C5A0C310C000001009F
:1064A0000101493CCAFBB6D2F6D8004422B68401A9
:1064B0006201AC008A02A302C302919093929537C5
:1064C000F1F4F5F6F76766363534979694E200E90D
:1064D00000EA00B500B600B700CD008301CC008A09
:1064E000019201940121022302240225022602279F
:1064F000022A02B300B4006F0070009F01CB019F1D
:1065000002A002E200E900EA00B500B600B700CD43
:10651000008301CC008A019201940121022302240C
:10652000022502260227022A02B300B4006F00707F
:0A653000009F01CB019F02A00200B2
:00000001FF
